:020000020000FC
:10000000FFC0E4C4E4C4E4C4FBC4FBC433C528C5D6
:1000100028C528C524C510C510C510C50AC50AC500
:100020000AC529C520C520C520C526C522C520C5AD
:0400300024C524C5FA
:10020000F89400E810E0009361001093610004E1AD
:1002100005B90FEE04B904E408B90FEB07B900EC17
:100220000BB90FE30AB9B1E0A0E0D5E0C0E000E00F
:100230000D93BD17E9F7AC17D9F714E00FEF1EBF08
:100240000DBF00E005BF03E00CBB00E105BB01E210
:1002500004BD0BE005BD00E006BD02E307BD00E004
:1002600008BD00E003BD00E00093800003E00093C0
:10027000810000E00093820010E000E01093850010
:100280000093840010E000E0109389000093880040
:1002900010E000E010938B0000938A0010E000E073
:1002A000109387000093860000E107BB01E20093F2
:1002B000B0000CE00093B10000E00093B20002E354
:1002C0000093B30000E00093B40000E00093B60098
:1002D00006EE00937C0005EE00937A0000E00093A8
:1002E0007B0000E000937E0000E80093300000E017
:1002F00000937F0010E003E01093C5000093C4005A
:1003000002E20093C00000E00093C10006E0009309
:10031000C20000E000937B0001E000936900A89513
:1003200008E10093600009E20093600002E8009396
:10033000640001E00DBB05E00093680000E100935C
:100340006B0000E000936C0000E800936D0000E09B
:1003500000936E0001E000936F0000E000937000D6
:100360000AE0202E0AE0402E04E60093100106E980
:100370000093110106E90093120108EC00931301A8
:1003800004E6009330010DE70093310106E9009384
:10039000320108EC0093330108E20093550100910B
:1003A000120100931A0100931B0100913201009386
:1003B0003A0100933B010AE00093600190E081E183
:1003C000D1D30F3FB1F00093110182E1CBD3009361
:1003D000120180E3C7D30093300181E3C3D30093BC
:1003E000310182E3BFD30093320183E3BBD3009397
:1003F0003301789406E9A89591FFFDCF9D7F0A957A
:10040000D1F704B700FF0EC00E7F04BF1AEFA89506
:1004100091FFFDCF9D7F1A9509F460C200913A01CA
:100420000A3AA8F70091330110913201011B0093A1
:1004300036010091320110913001011B009334010B
:100440000091320110913101011B08F400E000938A
:1004500035010091130110911201011B0093160147
:100460000091120110911001011B0093140102E888
:1004700000935201A89591FF30C29D7F429893FD51
:1004800017C0109132012091320136E0131B230F67
:1004900000913A010CD320F40AE0009360011DC2E0
:1004A000009160010A950093600109F016C29860FE
:1004B00002E0402E9F7E00911A0110911B01011B4A
:1004C00099F008F408C023E0033008F421E0120F8B
:1004D00010931B0109C0019523E0033008F421E0CB
:1004E000121B10931B0100C000913A0110913B01B7
:1004F000011B99F008F408C023E0033008F421E060
:10050000120F10933B0109C0019523E0033008F45A
:1005100021E0121B10933B0100C092FD17C0009117
:1005200078000091790010915201011720F008E243
:100530000093550122C0009155010A950093550181
:1005400021F408E200935501946017C000917800EF
:100550000091790010915201011720F408E20093F4
:1005600055010BC0009155010A950093550121F4E6
:1005700008E2009355019B7F00C092FF01C0A9C112
:1005800000911B0110911201011B00931C010091AD
:100590003B0110913201011B00933C0100913C0191
:1005A00007FD81C0065008F41EC19F7D05B100FD06
:1005B00002C00FEFE1D2589A289A009136010093B9
:1005C000B30007BD00911C0107FF19C000911C0179
:1005D000019510913C0120911601A9D210913C0186
:1005E000010F109113013091110120911201321B62
:1005F000230F121B209116019AD28FD21BC000919B
:100600001C0110913C012091160191D2102F0091F4
:100610003C01011B08F400E010911301309111011D
:1006200020911201321B230F121B209116017FD241
:1006300074D200C000911C0107FF1CC000911C0176
:10064000019510913C012091140171D2102F00915D
:100650003C01011B08F400E02091100130911101D0
:1006600010911201311B130F121B209114015FD244
:100670004CD218C000911C0110913C012091140132
:1006800056D210913C01010F2091100130911101BF
:1006900010911201311B130F121B2091140147D22C
:1006A00034D200C01AC100913C010195065008F4F3
:1006B0009AC09F7D05B100FF02C00FEF5DD2589830
:1006C0002898009134010093B30007BD00911C01EC
:1006D00007FF20C000911C01019510913C0111956C
:1006E0002091160124D210913C011195010F109117
:1006F0003501209134011BD2109113013091110169
:1007000020911201321B230F121B209116010FD2D0
:1007100004D222C000911C0110913C01119520913E
:10072000160105D210913C011195101B08F410E040
:10073000012F1091350120913401F9D1109113014D
:100740003091110120911201321B230F121B2091B5
:100750001601EDD1E2D100C000911C0107FF23C0BA
:1007600000911C01019510913C01119520911401FB
:10077000DED110913C011195101B08F410E0012FFF
:100780001091350120913401D2D120911001309186
:10079000110110911201311B130F121B2091140132
:1007A000C6D1B3D11FC000911C0110913C0111951D
:1007B00020911401BCD110913C011195010F1091B1
:1007C000350120913401B3D12091100130911101F4
:1007D00010911201311B130F121B20911401A7D18C
:1007E00094D100C07AC0109112012091120136E01C
:1007F000131B230F00911B015AD108F401C0906212
:1008000095FF67C0109112012091120136E0131B71
:10081000230F00911B014BD108F05BC000911C011C
:1008200007FD2BC005B100FD02C00FEFA5D1589800
:10083000289A109116011093B30000911C01209189
:10084000100110911101121B2091140170D15DD182
:10085000109116011093B30000911C011091350105
:100860002091340164D11091130120911101121BC8
:10087000209116015CD151D130C005B100FF02C0FA
:100880000FEF7AD1589A28981091140117BD009152
:100890001C0101951091130120911101121B20914F
:1008A000160145D13AD1109114011093B300009173
:1008B0001C010195109135012091340138D120910E
:1008C000100110911101121B2091140130D11DD182
:1008D00004C000E008BD0093B400CCCD13E004E6F2
:1008E0004BD11A95E1F700913A0100933301009141
:1008F0001A010093120142980AEF3ED1429A12E384
:1009000004E63AD11A95E1F710E527E800913A019B
:1009100000933001CCD008F451C042980AEF2CD19A
:10092000429A12E304E628D11A95E1F700913A01C0
:100930000093320142980AEF1FD1429A12E304E673
:100940001BD11A95E1F700913A01009331014298C9
:100950000AEF12D1429A12E304E60ED11A95E1F79A
:1009600000911A01009311013AE010913301209196
:100970003301131B230F00913A0199D008F41EC0D4
:1009800075EA0091110181E1DED00091120182E14E
:10099000DAD00091300180E3D6D00091310181E3BB
:1009A000D2D00091320182E3CED00091330183E3B3
:1009B000CAD070E042980AEFDFD0FCCF70E04298D6
:1009C00006E4DAD0429A06E4D7D0F8CF1895189505
:1009D000FFB60F931F93009184001C9903C00093EE
:1009E00038010AC00093390110913801011B02330C
:1009F00018F000933A0192601F910F91FFBE189575
:100A00001895FFB60F931F93009184004F9903C070
:100A1000009318010AC00093190110911801011BDD
:100A2000023318F000931A0191601F910F91FFBEDD
:100A3000189518951895189518951895FFB64A9415
:100A400061F490610F93429A00911A0100931B0187
:100A500000E008BD0093B4000F91FFBE18951895F3
:100A6000189518951895189518951895189518951E
:100A7000189518951895189518951895189510E0CB
:100A800010937A0010917C00107F102B10937C0043
:100A900000E000937B0005EC00937A0000917A005F
:100AA00006FDFCCF009178001091790008950117A0
:100AB00010F0201700F008956F937F93712F602F2F
:100AC000621B730B28F0712F602F461B570B00F031
:100AD0007F916F9108954F935F936F9344275527AC
:100AE00060E1000F111F441F551F4217530718F0F4
:100AF0000395421B530B6A95A1F75F934F932F9178
:100B00003F916F915F914F9108951F9317B5011712
:100B100008F0012F08BD1F9108951F931091B30095
:100B2000011708F0012F0093B4001F9108950F9250
:100B30001F923F93019F112D002D30E0CCDF3F919C
:100B40001F900F9008951F93F999FECF10E01FBBDF
:100B500010E012BD81BD00BD753A11F4FA9AF99A00
:100B60001F9108951F93F999FECF10E012BD81BD2A
:100B7000F89A00B51F9108951F932F93A8952AE026
:100B800015ED1A95F1F72A95D9F70A95B9F72F912E
:040B90001F91089514
:00000001FF
